:102319002020202020202020202020200D0A002AF3
:102329004D3A2053656C6674657374206F6B0D0AA2
:10233900002A573A2053656C667465737420666188
:10234900696C65640D0A002A52454144590D0A0019
:1023590000022F002F2A00AB20015E1601D21102C4
:102369005A0C02780B02960A02B60902D70802F93A
:1023790007031C06033F05036404038B0303B2022E
:0623890003DA0104040068
:10144E00906F147401F0906F14E0FD64126024ED3F
:10145E0075F003A42459F582E43423F583E493FA5A
:10146E00740193FBC3EF9BEE9A4008906F14E00457
:10147E00F080D3ED75F003A42459F582E43423F5FE
:10148E0083C37401939FFFE4939EFEE4FCFD7BE80F
:10149E007A03F9F81204EDC8ECC8C9EDC9CAEECA50
:1014AE00CBEFCB906F14E0FF75F003A4245BF582B5
:1014BE00E43423F583E493FDEF75F003A42458F58B
:1014CE0082E43423F583E493C39DFFE49400FEE4A9
:1014DE00FCFD1204EDECC0E0EDC0E0EEC0E0EFC0AC
:1014EE00E0906F14E0FF75F003A42456F582E43407
:1014FE0023F583E493FC740193FDEF75F003A424AC
:10150E0059F582E43423F583C37401939DFFE4936C
:10151E009CFEE4FCFDF8F9CAEECACBEFCBD0E0FF9F
:10152E00D0E0FED0E0FDD0E0FC120578EEC0E0EF9A
:10153E00C0E0906F14E075F003A4245BF582E434F0
:10154E0023F583E493FFE4FCFDFE7BE87A03F9F8D0
:0C155E001204EDD0E02FFFD0E03EFE2292
:10222900201175906F73E05407906F0BF0C39403FE
:102239004066E064076061D2117F0112307DE4904D
:102249006F0BF07F017D127B03123147301706E5D2
:102259006860F980397F017D0E7B031231473017A1
:1022690006E56860F980277F017D0A7B0212314704
:10227900301706E56860F98015906F0BE004F0E00F
:10228900B403C07F0112311C7F0A12307D227F0204
:0922990012311C7F0A12307D2273
:10130E003012030213E8E56864036009E568640BB4
:10131E00600302144DD378D5E6954F18E6954E40EE
:10132E000A906F12E4F0A304F0803BAF4FAE4E1262
:10133E00144EEEC0E0EFC0E078D4E6FE08E6FF12F1
:10134E00144ECCEECCCDEFCDD0E0FFD0E0FEC3ED11
:10135E009FFFEC9EFE906F12F0A3EFF04E70079081
:10136E006F12F0A304F0D201E4906F0BF0906F12A5
:10137E00E0FAA3E0FB7C007D0AFFCEEACE12043633
:10138E00906F0BE0240CF582E4346FF583EDF07C66
:10139E00007D0ACFEBCFCEEACE120436906F12EE5E
:1013AE00F0A3EFF0906F0BE004F0E0B405BF906F88
:1013BE000B7404F0906F0BE0FFF46015740C2FF5B6
:1013CE0082E4346FF583E07008906F0BE014F080C8
:1013DE00E3EF04906F11F0D212227F1E12307D7F48
:1013EE00017D327B041231473017043016FA227F0A
:1013FE000A12307D906F11E014906F0BF0906F0B0E
:10140E00E0240CF582E4346FF583E0700B7F017DF0
:10141E000B7B041231478016906F0BE0240CF58283
:10142E00E4346FF583E0FF7D0B7B011231473017FB
:10143E00043016FA22906F0BE0FF14F0EF70BE220C
:1020A800D2AF122F451230A012000E122F78123123
:1020B800811230F612000312212F1230047BFF7AAE
:1020C8002379191200C91230EC122B8950107BFFAA
:1020D8007A2379281200C97F0112311C800B7BFFFB
:1020E8007A23793A1200C9D211122014906EE7E0CF
:1020F800FF122B17122BC2122863906EE8E0FEA382
:10210800E0FF122A1A7BFF7A2379501200C9C21203
:10211800C211301603122EBA12130E906EDFE06051
:07212800F112222980EC22D4
:03000B0002238F3E
:10238F00C0E0C0F0C083C082C0D075D008C28CAF8F
:10239F008CEFFEAD8AED255F78D7F6E55E3E18F639
:1023AF00F58C08E6F58AD28CD56309906EDEE0F5E0
:1023BF006312273FD5621B906EDEE0F5620561E583
:1023CF006170020560E56145607007E5686003753F
:1023DF006805E5686404600F121888122618121E2B
:1023EF0019122CCE121F77D0D0D082D083D0F0D03C
:0223FF00E032CA
:102A1A00E4FCFDFB7AC079A8F81204ED7BE07A2E7B
:102A2A00790078001229D6C374129FF55FE49EF5E7
:102A3A005E906EDEE0F563F562E4F560F561E589C6
:102A4A0054F04401F589758CFF758AFFC2B9D2A981
:032A5A00D28C22F9
:0C30BC00906EDEE0F562E4F560F5612244
:10286300E5C520E3FB75C50775C50FE5C530E4FB7A
:10287300AFC6EF75F004A4FFAEF0E5C5C41313545F
:10288300037C002FF53CEC3EF53BE4F53AE53A25B5
:10289300E024C0F8A63B08A63CE53C2527F527E540
:1028A3003B3526F526053AE53AB40AE1E4F5392243
:10188800C0D075D008E5C520E3FBE4F5C575C508EB
:10189800F543754401E5436408700302195DE5C525
:1018A80030E4FB85C62885C53DE5436407600EE541
:1018B800C520E3FBE54304F5C54408F5C5E52875EF
:1018C800F004A4FFAEF0E53DC4131354037C002FCD
:1018D800F546EC3EF545E54325E02429F8A64508FC
:1018E800A646906EDDE055446060AF28122BF9AF34
:1018F8003D122BF9E543B4060885454185464280EB
:1019080049E54364077043E53925E024C1F8C3E598
:101918002796F527E5261896F526E53925E024C00B
:10192800F8A64508A646E5462527F527E5453526C0
:10193800F526FEAF277C007D0A1204368E248F25FB
:101948000539E539B40A03E4F5390543E54425E0EA
:10195800F54402189D300F1EE4A2C492E4A2C59279
:10196800E5A29692E6A29792E72568C4F53EAF3EB7
:0D197800122BF9853E40C294D294D0D022AB
:10240100C0D075D008300F65906EE7E0FD7C00907C
:102411006EF2E0FB24FFFFE434FFFE120422EF24FE
:1024210001FFE43EFEC3E51F9FF51FE51E9EF51E5D
:102431008B3FE53F6021E51EF583E51FF582E0C492
:1024410054F02568C4F0906EE7E0251FF51FE435D0
:102451001EF51E153F80DB906EE7E024FFFFE4349C
:10246100FFFEC3E51F9FF51FE51E9EF51ED0D0227E
:0D30AF00E4F576F577F578C219122B502262
:10261800C0D075D008E568605720195412306A4058
:102628004F906EE7E02404906F05F0906F05E0602E
:102638003F20133C122C9A8F7512002E0577E577F0
:10264800700205767004E5766480701CF576F5777F
:102658000578E578B40C04D2198015123057E5785E
:1026680020E005122B508008906F05E014F080BB25
:03267800D0D0229D
:102BC200E4906FB2F0906EF2E075F00584906FB110
:102BD200F0E4906FB3F0906FAD1206500000000069
:102BE20074FF78D4F608F6E4906FB4F0F569F568EE
:072BF200906FAC74FFF022AC
:102F2B00C0D075D008756801AF68122FA8C2901277
:0A2F3B0030AF7F0212311CD0D0220B
:102FD800C0D0C291E5612401906FABF0E4356090F8
:062FE8006FAAF0D0D02218
:102FEE00C0D0C292E5612401906FABF0E4356090E1
:062FFE006FAAF0D0D02202
:1011B000C0D075D008E4906F05F020C604E044016B
:1011C000F020C707906F05E04402F0906FACE0FF9D
:1011D000906F05E0FE6F603BEE7025906FBAE0FF08
:1011E0006005123124802C906FB9E0FF6403600425
:1011F000EFB40405123124801A7F0112311C8013D0
:10120000906F05E030E0077F0112312480057F02F6
:10121000123124906F05E0906FACF0300B1EA29459
:10122000300C01B34016C21A1230BC906EDBE0FEE7
:10123000A3E0FF122CFE122F2B02130B201003022F
:10124000130B906EDAE0C4F8540FC868FF906ED9A3
:10125000E0C454F048FEC3E54D9FFDE54C9EFCE51F
:1012600042C4F8540FC868FFE541C454F048FED3A7
:10127000EF9DEE9C402A906FB1E014F07028D21AD6
:10128000906FAD12065000000000E4906FB2F09035
:101290006EF2E075F00584906FB1F01230BC806B97
:1012A000906FB1E004F0C21A906FADE0F8A3E0F9DE
:1012B000A3E0FAA3E0FBE8C0E0E542C4F8540FC89D
:1012C00068FFE541C454F048FEC3EF954DFFEE952D
:1012D0004CFE3395E0FDFCD0E0F8EB2FFFEA3EFE3C
:1012E000E93DFDE83CFC906FAD120644906EF2E0E3
:1012F000FF906FB2E004F06F7011906EE2E0FEA319
:0E130000E0FF122CFE122F2B122401D0D0225F
:101ED200C0D075D008906FADE0F8A3E0F9A3E0FAA6
:101EE200A3E0FBE8C0E0E542C4F8540FC868FFE590
:101EF20041C454F048FEC3EF954DFFEE954CFE33BE
:101F020095E0FDFCD0E0F8EB2FFFEA3EFEE93DFD57
:101F1200E83CFC906FAD120644300E387F007E0024
:101F22007D007C00906FADE0F8A3E0F9A3E0FAA396
:101F3200E0FBD312060A401C906ED8E0FFD3E561A5
:101F42009FE5609400400D122FD8756802AF6812A9
:101F52002FA8801E300D1B906EEEE0FEA3E065619F
:101F62007003E5606E700B122FD875680AAF6812A5
:051F72002FA8D0D022D1
:1022A200C0D075D008906FAAE0FEA3E0656170030C
:1022B200E5606E7002D291300E3C906EE5E0FEA3B6
:1022C200E0FFC3E54F9FFFE54E9EFEC3E5259FE578
:1022D200249E5007E4906FB3F0801B906F03E0FFE1
:1022E200906FB3E004F06F700D122FEE756803AFBC
:1022F20068122FA8801E300D1B906EF0E0FEA3E046
:1023020065617003E5606E700B122FEE75680BAF9E
:0723120068122FA8D0D022B1
:102ED800C0D075D008906FAAE0FEA3E065617003CA
:0C2EE800E5606E7004D291D292D0D0222E
:101E1900C0D075D008E5687003021EA7E4F56475A3
:101E29006701E56464086065E56425E024F3F582EB
:101E3900E4346EF583E0FEA3E08E65F566F4700385
:101E4900E565F4603EE56955677015E5616566709D
:101E590004E56065657009E5674269AF641228FFAA
:101E6900E5695567601DE5662401FFE43565FEEF08
:101E790065617003EE6560700AE567F45269AF64E5
:101E890012298F0564E56725E0F5678095C3E52587
:101E990078D596E52418965005A62408A625E56860
:101EA90014601614601814601A24F9601114601370
:101EB900240B70121211B0800D121ED2800812224A
:091EC900A28003122ED8D0D02211
:102B1700CBEFCBEBFD7C007E3A7F98120436CDEBF2
:102B2700CD7C001204228E1A8F1B74002FF582EEC3
:102B37003434AF82F5188F197E347F008E1C8F1DB9
:092B47008E1E8F1FD213C214224E
:102BF900201933C213051FE51FAC1E7002051E14F0
:102C0900F5828C83EFF0E51F65197004E51E6518E0
:102C19007006751E34751F00E51F651D7004E51EDD
:072C2900651C7002D21422A9
:102C9A00C214051DE51DAE1C7002051C14F5828EBA
:102CAA0083E0FFE51D65197004E51C65187006755B
:102CBA001C34751D00E51F651D7004E51E651C703A
:042CCA0002D21322FD
:102CFE00C3E51F9FF51DE51E9EF51CC3E51D940043
:102D0E00E51C9434400BD3E51D9519E51C95184030
:0E2D1E000CE51B251DF51DE51A351CF51C22C4
:101C6C002573202562752025627520257520257524
:101C7C002025752025752025632025627520256378
:101C8C002025632025630D0A00632069676E2025DB
:101C9C007520257520257520257520257520257521
:101CAC002025752025750D0A006320786D69742038
:101CBC00257520256275202562750D0A0063206349
:101CCC0068616E202562750D0A00632067707320B1
:101CDC002562750D0A00696E646578006572617322
:101CEC0065006F6666006F6E002A56455253494F69
:101CFC004E3A20522D4441532056332E350D0A00B6
:101D0C0063210063207264617300632069676E0055
:101D1C006320786D69740063206368616E006320D2
:101D2C0067707300633F006300632000677073206B
:101D3C00007265736574002A453A20756E6B6E6F80
:091D4C00776E20636D640D0A003E
:08000300E4F57EC216C21522CD
:100AF600906F0BEBF0A3EAF0A3E9F0300B13300C88
:100B060008906F287401F0800D906F287402F080B1
:100B160005E4906F28F0906F0BE0FBA3E0FAA3E0EA
:100B2600F91203BA643F6003020BDC906F0EE0F922
:100B3600A3E0FAA3E0906F33C9F0A3EAF0A3E9F0CB
:100B4600906EDEE0906F36F0906EDDE0906F37F0DD
:100B5600906ED9E0FFA3E0906F38CFF0A3EFF0904E
:100B66006EE5E0FFA3E0906F3ACFF0A3EFF0906E52
:100B7600EEE0FFA3E0906F3CCFF0A3EFF0906EF0B5
:100B8600E0FFA3E0906F3ECFF0A3EFF0300F047FBD
:100B96003180027F30906F40EFF0906F28E0906FC9
:100BA60041F03010047F3180027F30906F42EFF0C9
:100BB600300E047F3180027F30906F43EFF0300DAE
:100BC600047F3180027F30906F44EFF07BFF7A1C08
:100BD600796C1200C922906F0BE0FBA3E0FAA3E048
:100BE600F91203BAFF12301A500C906F0CE475F02C
:100BF600011204C180E0E4906F27F0906F0BE0FBD8
:100C0600A3E0FAA3E0F9121678906F27E025E02416
:100C160011F582E4346FF583EEF0A3EFF0906F0BDD
:100C2600E0FBA3E475F0011204D7A9F0FA1203BAA7
:100C3600FF12301A50E7906F27E004F0E0B40BBBC8
:100C4600906F12E0906EDEF0906F14E0906EDDF023
:100C5600906F15E0FFA3E0906ED9CFF0A3EFF09070
:100C66006F17E0FFA3E0906EE5CFF0A3EFF0906F73
:100C760019E0FFA3E0906EEECFF0A3EFF0906F1BAC
:100C8600E0FFA3E0906EF0CFF0A3EFF0906F1DE0D1
:100C9600FEA3E0FFEE4F24FF920FA3E0FEA3E0FFCA
:100CA600EE4F24FF920BEF64014E7003D38001C315
:100CB600920C906F21E0FEA3E0FFEE4F24FF92100E
:100CC600A3E0FEA3E0FFEE4F24FF920EA3E0FEA3F7
:090CD600E0FFEE4F24FF920D2215
:10178600906F0BEBF0A3EAF0A3E9F01203BA643F03
:10179600600302181D7BFF7A1C7995906EF3E0FFBB
:1017A600A3E0906F33CFF0A3EFF0906EF5E0FFA3C8
:1017B600E0906F35CFF0A3EFF0906EF7E0FFA3E077
:1017C600906F37CFF0A3EFF0906EF9E0FFA3E090B3
:1017D6006F39CFF0A3EFF0906EFBE0FFA3E0906FC0
:1017E6003BCFF0A3EFF0906EFDE0FFA3E0906F3DDE
:1017F600CFF0A3EFF0906EFFE0FFA3E0906F3FCF36
:10180600F0A3EFF0906F01E0FFA3E0906F41CFF0FF
:10181600A3EFF01200C922906F0BE0FBA3E0FAA33E
:10182600E0F91203BAFF12301A500C906F0CE475EF
:10183600F0011204C180E0E4906F0EF0906F0BE0AF
:10184600FBA3E0FAA3E0F9121678906F0EE025E00C
:1018560024F3F582E4346EF583EEF0A3EFF0906F97
:101866000BE0FBA3E475F0011204D7A9F0FA12030A
:10187600BAFF12301A50E7906F0EE004F0E0B40899
:02188600BB2283
:101D5500906F0BEBF0A3EAF0A3E9F01203BAB43FDE
:101D6500297BFF7A1C79B5906EE0E0FFA3E0906FC8
:101D750033CFF0A3EFF0906EEAE0906F35F0906FFF
:101D850004E0906F36F01200C922906F0BE0FBA3C0
:101D9500E0FAA3E0F91203BAFF12301A500C906F63
:101DA5000CE475F0011204C180E0E4906F14F0902A
:101DB5006F0BE0FBA3E0FAA3E0F9121678906F141D
:101DC500E025E0240EF582E4346FF583EEF0A3EF11
:101DD500F0906F0BE0FBA3E475F0011204D7A9F0B6
:101DE500FA1203BAFF12301A50E7906F14E004F0AC
:101DF500E0B403BB906F0EE0FFA3E0906EE0CFF080
:101E0500A3EFF0906F11E0906EEAF0906F13E09001
:041E15006F04F02244
:10267B00906F0BEBF0A3EAF0A3E9F0906F0BE0FB8C
:10268B00A3E0FAA3E0F91203BAB43F127BFF7A1C62
:10269B0079C9906EEDE0906F33F01200C922906F04
:1026AB000BE0FBA3E0FAA3E0F91203BAFF12301A16
:1026BB00500C906F0CE475F0011204C180E0906F28
:1026CB000BE0FBA3E0FAA3E0F9121678906EEDEFA6
:0226DB00F022EB
:1026DD00906F0BEBF0A3EAF0A3E9F0906F0BE0FB2A
:1026ED00A3E0FAA3E0F91203BAB43F127BFF7A1C00
:1026FD0079D6906EDFE0906F33F01200C922906FA3
:10270D000BE0FBA3E0FAA3E0F91203BAFF12301AB3
:10271D00500C906F0CE475F0011204C180E0906FC5
:10272D000BE0FBA3E0FAA3E0F9121678906EDFEF51
:02273D00F02288
:1006F9007B017A6E799A7D20122EF4906F0EEBF0C1
:10070900A3EAF0A3E9F04A70047F0180027F009018
:100719006F1BEFF0605F7B017A6E7999121678C8CA
:10072900ECC8C9EDC9CAEECACBEFCB906EEBE0FEBF
:10073900A3E0FFE4FCFD1204EDC8ECC8C9EDC9CA89
:10074900EECACBEFCB906EDBE0FEA3E0FFE4FCFD4D
:10075900EB2FFFEA3EFEED39FDEC38FC906F1112EC
:100769000644906EEBE0FEA3E0FFE4FCFD906F15FC
:1007790012064480767B017A6E7999121678C8EC54
:10078900C8C9EDC9CAEECACBEFCB906EE7E0FFE46A
:10079900FCFDFE1204EDC8ECC8C9EDC9CAEECACB0E
:1007A900EFCB906EDBE0FEA3E0FFE4FCFDEB2FFF57
:1007B900EA3EFEED39FDEC38FC906F1112064490CB
:1007C9006F0EE0FBA3E0FAA3E0F9121678C8ECC8B3
:1007D900C9EDC9CAEECACBEFCB906EE7E0FFE4FCE6
:1007E900FDFE1204ED906F15120644906F11E0FCA6
:1007F900A3E0FDA3E0FEA3E0FF780F1206318F7896
:10080900906F11E0FCA3E0FDA3E0FEA3E0FFEE542E
:100819007FFEE48E768F77123057906F1BE0600968
:10082900E4906F19F0A3F0800B120026906F19EE77
:10083900F0A3EFF0E4906F0BF0A3F0906F0BE0FEE4
:10084900A3E0FFE4FCFD906F15E0F8A3E0F9A3E055
:10085900FAA3E0FBC3120620606C1230C8906F0D3A
:10086900EFF0906F1BE06014906F0DE0FF906F1A2E
:10087900E02FF0906F19E03400F08018906F19E0C4
:10088900FEA3E0FF906F0DE0FD1221AD906F19EE10
:10089900F0A3EFF0906F0DE0FF1231140577E577C3
:1008A900700205767004E57664807009F576F5774F
:1008B9000578123057906F0CE004F07006906F0BBA
:1008C900E004F0020844906F1BE07013906F19E088
:1008D900FEA3E0FF12313A906F19EEF0A3EFF0900A
:1008E9006F19E0FF123114906F1AE0FF12311422D0
:10302F00D3EF648094B95007EF24D0FEFF8004EFF4
:04303F0024A9FF229F
:10198500906F0BEBF0A3EAF0A3E9F0906F1274FFF0
:10199500F0A3741CF0A374E2F0A3E4F0A37405F0C3
:1019A5001225B1EF7003122947906F1274FFF0A34F
:1019B500741CF0A374E8F0A3E4F0A37405F0906F31
:1019C5000BE0FBA3E0FAA3E0F91225B1EF700412D6
:1019D5002F5F22906F1274FFF0A3741CF0A374EEB6
:1019E500F0A3E4F0A37403F0906F0BE0FBA3E0FA1F
:1019F500A3E0F91225B1EF7003C21522906F12749E
:101A0500FFF0A3741CF0A374F2F0A3E4F0A3740236
:101A1500F0906F0BE0FBA3E0FAA3E0F91225B1EF1C
:101A25007003D21522906F0BE0FBA3E0FAA3E0F957
:101A35001203BAFF122DA95043906F0BE0FBA3E0F0
:101A4500FAA3E0F99000011203D3FF12302FCDEF76
:101A5500CD906F0BE0FBA3E0FAA3E0F91203BAFF08
:101A650012302FEFC454F02DFF906F0EF0122F900F
:0D1A7500906F0CE475F0021204C180A922EC
:04317100122E1822E0
:0A30EC007BFF7A1C79F51200C9225F
:1008F900906F1274FFF0A3741DF0A3740CF0A3E4BD
:10090900F0A37402F07B017A6E79981225B1EF7029
:1009190004120CDF22906F1274FFF0A3741DF0A370
:10092900740FF0A3E4F0A37406F07B017A6E799852
:100939001225B1EF7018906F0E74FFF0A3741DF0BB
:10094900A3740FF07B017A6E799E120AF622906FDA
:100959001274FFF0A3741DF0A37416F0A3E4F0A3BE
:100969007405F07B017A6E79981225B1EF700A7BD4
:10097900017A6E799D12178622906F1274FFF0A387
:10098900741DF0A3741CF0A3E4F0A37406F07B01BA
:100999007A6E79981225B1EF700A7B017A6E799E89
:1009A900121D5522906F1274FFF0A3741DF0A374E9
:1009B90023F0A3E4F0A37406F07B017A6E79981210
:1009C90025B1EF700A7B017A6E799E12267B2290FF
:1009D9006F1274FFF0A3741DF0A3742AF0A3E4F05E
:1009E900A37405F07B017A6E79981225B1EF700A2C
:1009F9007B017A6E799D1226DD22906F1274FFF0C9
:100A0900A3741DF0A37430F0A3E4F0A37402F07B87
:100A1900017A6E79981225B1EF7018906F0E74FFF4
:100A2900F0A3741DF0A37433F07B017A6E799912E7
:100A39000AF622906F1274FFF0A3741DF0A37435A7
:100A4900F0A3E4F0A37402F07B017A6E7998122581
:100A5900B1EF7018906F0E74FFF0A3741DF0A374BA
:100A690033F07B017A6E7999120AF622906E98E03A
:100A7900B464041206F922906F1274FFF0A3741D76
:100A8900F0A37438F0A3E4F0A37404F07B017A6E48
:100A990079981225B1EF700A7B017A6E799C121947
:100AA9008522906F1274FFF0A3741DF0A3743DF0BA
:100AB900A3E4F0A37405F07B017A6E79981225B14D
:100AC900EF700412317122906E98E0B46904121A21
:100AD9008222906E98E0B476041230EC22906E98DF
:0D0AE900E060097BFF7A1D79431200C922ED
:102EBA0010160280107568047F0112311C7F1E12E1
:0E2ECA00307D1208F93015E81227A180E322AE
:102C3000C0D0EF20E72CEF640A6027EF640D60112D
:102C40007498257EF582E4346EF583EFF0057E807E
:102C5000117498257EF582E4346EF583E4F0D21683
:052C6000F57ED0D0223A
:102471002A4D4553534147453A2053746F72696E53
:102481006720706172616D657465727320696E2079
:10249100464C4153480D0A002A4D45535341474587
:1024A1003A2046696E69736865642073746F726956
:1024B1006E670D0A00000001C001C802000C001B7C
:1024C10001000019003C03FFFFFFFFFFFFFFFFFFBB
:0D24D100FFFFFFFFFFFFFF00000A010000FA
:0A30F600757C24757DB612102922A6
:101029009024B6E49324FF920BA3E49324FF920C3B
:10103900A3E49324FF9210A3E493906EDDF090242F
:10104900BAE49324FF920FE4906EE7F07F80EF609B
:1010590014906EDDE05F6007906EE7E02402F0EF28
:10106900C313FF80E9300F06906EE7E004F0902487
:10107900BBE493906EDEF09024BCE493906EE4F0B0
:101089009024BDE493FF740193906ED9CFF0A3EF40
:10109900F09024BFE493FF740193906EE5CFF0A321
:1010A900EFF0906EDEE0FBFD7C007E037FE812042A
:1010B90036906EE8EEF0A3EFF0906EE7E0FA8BF071
:1010C900A4FF906EEBE5F0F0A3EFF0EB1313543FA0
:1010D900906EF2F0FB906F03F09024C1E49324FF2B
:1010E900920EA3E49324FF920DA3E493FF7401935A
:1010F900906EEECFF0A3EFF09024C5E493FF740156
:1011090093906EF0CFF0A3EFF09024C7E493906E24
:10111900D8F0906EE4E0FF7E00906EEBE0FCA3E077
:10112900FD120422906EDBEEF0A3EFF0EBFF7E00E0
:10113900EAFD7C00120422E02F906EE3F0906EDB52
:10114900E03E906EE2F0E4FFEF25E024C8F582E48A
:101159003424F583E493FC740193FDEF25E024F333
:10116900F582E4346EF583ECF0A3EDF00FEFB408EB
:10117900D79024D8E493FF740193906EE0CFF0A345
:10118900EFF09024DAE493906EEAF09024DBE49394
:10119900906F04F09024DCE493906EEDF09024DDE0
:0711A900E493906EDFF022D9
:100CDF00A20BE433857D82857C83F0A20CE433A3E1
:100CEF00F0A210E433857D82857C83A3A3F0906E00
:100CFF00DDE0857D82857C83A3A3A3F0A20FE4337F
:100D0F00FFE57D2404F582E4357CF583EFF0906EEA
:100D1F00DEE0FFE57D2405F582E4357CF583EFF019
:100D2F00906EE4E0FFE57D2406F582E4357CF583E3
:100D3F00EFF0906ED9E0FEA3E0FFE57D2407F5828A
:100D4F00E4357CF583EEF0A3EFF0906EE5E0FEA3C3
:100D5F00E0FFE57D2409F582E4357CF583EEF0A311
:100D6F00EFF0A20EE433FFE57D240BF582E4357C32
:100D7F00F583EFF0A20DE433FFE57D240CF582E45B
:100D8F00357CF583EFF0906EEEE0FEA3E0FFE57D9E
:100D9F00240DF582E4357CF583EEF0A3EFF0906E31
:100DAF00F0E0FEA3E0FFE57D240FF582E4357CF54E
:100DBF0083EEF0A3EFF0906ED8E0FFE57D2411F500
:100DCF0082E4357CF583EFF0E4906F0BF0906F0BBE
:100DDF00E0FF6408603BEF25E024F3F582E4346E16
:100DEF00F583E0FEA3E0FFE57D2412F582E4357C78
:100DFF00F583C083C082906F0BE0D082D08375F0F3
:100E0F0002120681EEF0A3EFF0906F0BE004F0807A
:100E1F00BC906EE0E0FEA3E0FFE57D2422F582E4C6
:100E2F00357CF583EEF0A3EFF0906EEAE0FFE57D01
:100E3F002424F582E4357CF583EFF0906F04E0FF16
:100E4F00E57D2425F582E4357CF583EFF0906EED9A
:100E5F00E0FFE57D2426F582E4357CF583EFF09005
:100E6F006EDFE0FFE57D2427F582E4357CF583EF27
:100E7F00F07BFF7A2479711200C9122C657BFF7AFF
:070E8F002479991200C92229
:10201400E5C520E3FB75C50675C50EE5C530E4FBD3
:10202400AFC6EF75F004A4FFAEF0E5C5C4131354B6
:10203400037C002FF54DEC3EF54CE5C520E3FB7524
:10204400C50775C50FE5C530E4FBAFC6EF75F004F1
:10205400A4FFAEF0E5C5C4131354037C002FF54A66
:10206400EC3EF549F54E854A4FD21AE4F547F5485A
:10207400FFEF25E0247AF582E4346FF583E54CF034
:10208400A3E54DF0E54D2548F548E54C3547F547C2
:102094000FEFB410DCE4F54BE5482401F54DE435CD
:0420A40047F54C228E
:10273F00301A5EE5482401F54DE43547F54CE54B7D
:10274F0025E0247AF582E4346FF583E0FEA3E0FF01
:10275F00C3E5489FF548E5479EF547E54B25E0243F
:10276F007AF582E4346FF583E541F0A3E542F0E5B5
:10277F00422548F548E5413547F547054BE54BB44C
:10278F001003E4F54B85494E854A4F85244985252D
:02279F004A22CC
:102F4500D21B43878075985AE589540F4420F5892B
:0A2F5500758DFFD28ED2BCD2AC22E3
:03002300022D5754
:102D5700C0E0C0F0C083C082C0D075D010309807E3
:102D6700AF99C298122C30309904C299D21BD0D097
:092D7700D082D083D0F0D0E0320C
:08311400301BFDC21B8F992244
:07312C00CEEFCE1231142298
:102D8000E5C520E3FB8FC5EF4408F5C5E5C530E494
:102D9000FBAFC6EF75F004A4FFAEF0E5C5C4131396
:092DA0005403FDE5F0EF4DFF22A4
:102E1800E4F5A8F5E8F5B8F5F875780FE578A2E0D7
:102E280092B5A2E192B3A2E292B4A2E392B202FFF7
:022E3800FE2278
:10305700E578A2E092B5A2E192B3A2E292B4A2E32C
:0330670092B22200
:0C30C800E5764480857782F583E0FF22E6
:10002E0090D3557499F090ACAA7466F090D3557431
:10003E0090F0E575F5F0E576D2E7F583E577F58294
:0D004E00E5F0F0E0A2E730F701B340F72243
:102B5000E578A2E092B5A2E192B3A2E292B4A2E338
:102B600092B290D3557499F090ACAA7466F090D359
:102B7000557480F090D3557499F090ACAA7466F0B7
:092B80009080007414F0D21C22B4
:10306A00301C0D908000E020E703D38001C3921C3E
:03307A00A21C2273
:102C650075780C122B5012306A40FB75780D1230B6
:102C750057E4F576F577857782857683E0F57512E5
:102C8500002E0577E57770020576E5777004E57621
:052C9500648070E222E2
:03318100C21C224B
:03005B000224DE9E
:1024DE00C0E0C0D0C2CC742D25C9F5C9301758152F
:1024EE0050E5507052E55670128552FCC2C0F5513F
:1024FE00755601E55425E0F550803CE556640170B3
:10250E002375FCFFD2C00551E5516553700E30188E
:10251E0007F556855550801FC217801B75560275DC
:10252E0050028013E556B4020E8552FCC2C0755699
:0C253E0001E55425E0F550D0D0D0E0328B
:102F780075FCFFD2C075FE0B75528075EA0DC2FC58
:082F8800D2EC75550AC21722B4
:102DD200C217A202921875FCFFD2C08F53E4F556B7
:102DE200CEEDCE8EFECEEBCE8E54855550EF6002E8
:032DF200D21722D3
:06314100D202122DD22281
:06314700C202122DD2228B
:08311C007D0B7B011231412201
:083124007D327B0412314122CF
:10307D00C21775FCFFD2C08F55E4F556855550D259
:02308D00172208
:10156A00413A2534752025347520253475202534D3
:10157A0075202534752025347520253475202534A9
:10158A007520443A25303262782043433A25632550
:10159A00632042573A25630D0A002A4D3A20615FBB
:1015AA007374203D2025750D0A002A4D3A206128C2
:1015BA003029203D2025750D0A002A573A20615FFF
:1015CA0073743D25752C2061303D25752028672DC3
:1015DA0073772064697361626C6564290D0A002A55
:1015EA004D3A2070283029203D2025750D0A002A01
:1015FA00573A20502072616E6765205B25752C254D
:10160A00755D0D0A002A573A204257206572726F9B
:10161A0072202842572064697361626C6564290DDF
:10162A000A002A573A206E6F2069676E2025626485
:10163A000D0A002A573A206E6F20786D69740D0AD8
:10164A00002A573A206E6F206770730D0A002A57D6
:10165A003A2064726F677565206572720D0A002AF6
:0E166A00573A206D61696E206572720D0A009C
:07313300EF60031F80FA2288
:101A82001016028003021B79E4A2C492E0A2C5925E
:101A9200E1A29692E2A29792E3F57BE4FF122D80F7
:101AA200EFC0E0EEC0E07F01122D80EFC0E0EEC09B
:101AB200E07F02122D80EFC0E0EEC0E07F03122D26
:101AC20080EFC0E0EEC0E07F04122D80EFC0E0EEB8
:101AD200C0E07F05122D80EFC0E0EEC0E07F06126D
:101AE2002D80EFC0E0EEC0E07F07122D80906F41A5
:101AF200EEF0A3EFF0906F3FD0E0F0A3D0E0F090D3
:101B02006F3DD0E0F0A3D0E0F0906F3BD0E0F0A3C7
:101B1200D0E0F0906F39D0E0F0A3D0E0F0906F37D2
:101B2200D0E0F0A3D0E0F0906F35D0E0F0A3D0E0A9
:101B3200F0906F33D0E0F0A3D0E0F07BFF7A15791C
:101B42006A906F43E57BF030C6047F6380027F6F4B
:101B5200906F44EFF030C7047F6380027F6F906F15
:101B620045EFF03094047F6F80027F63906F46EF01
:081B7200F01200C9021A8222E0
:102E9B00A2029293E4F579F57A7F78123133057AB1
:0F2EAB00E57A70020579E57A640A457970EB22C1
:100E9600E4906F10F0906F0BF0A3F0906F0FF0D20C
:100EA60002122E9B7F06122D80906F0CE02FF09081
:100EB6006F0BE03EF0C202122E9B906F0FE004F023
:100EC600E0B420DB906F0BE0FEA3E0FF7C007D200A
:100ED60012048B906F0BEEF0A3EFF07BFF7A15797F
:100EE600A4906F33EEF0A3EFF01200C9E4906F0DFB
:100EF600F0A3F0A3F07F06122D80906F0EE02FF086
:100F0600906F0DE03EF0906F0FE004F0E0B420E546
:100F1600906F0DE0FEA3E0FF7C007D2012048B9015
:100F26006F0DEEF0A3EFF07BFF7A1579B4906F3377
:100F3600EEF0A3EFF01200C9906F0DE0FEA3E0FF04
:100F4600906F0BE0FCA3E0FDC39FFFEC9EFEC3EF9A
:100F5600942DEE64809480502D7BFF7A1579C49091
:100F66006F33ECF0A3EDF0906F0DE0FFA3E0906F10
:100F760035CFF0A3EFF01200C97F06123124C2105C
:100F8600906F107406F0E4906F0BF0A3F0906F0F63
:100F9600F07F07122D80906F0CE02FF0906F0BE022
:100FA6003EF0906F0FE004F0E0B420E5906F0BE0A8
:100FB600FEA3E0FF7C007D2012048B906F0BEEF009
:100FC600A3EFF07BFF7A1579E9906F33EEF0A3EF8C
:100FD600F01200C9906F0BE0FEA3E0FFC3947DEE14
:100FE60064809482400BD3EF94DBEE64809483405C
:100FF6002C7BFF7A1579F9906F33EEF0A3EFF0A30F
:101006007402F0A3747DF0A37403F0A374DBF012F2
:1010160000C97F05123124906F107405F0906F108F
:03102600E0FF22C6
:101B7A00E4906F0BF0300B1EA294300C01B34016A8
:101B8A007BFF7A16790F1200C97F03123124C20B28
:101B9A00906F0B7403F0E4906F0CF0906F0CE0FF01
:101BAA006408606AEF25E024F3F582E4346EF58375
:101BBA00E0FCA3E0F47002ECF4604B1230D4401F56
:101BCA007F041231247BFF7A16792C906F0CE00483
:101BDA00906F33F01200C9906F0B7404F080279055
:101BEA006F0CE0FF1228B3401D7F041231247BFFE3
:101BFA007A16792C906F0CE004906F33F01200C9BA
:101C0A00906F0B7404F0906F0CE004F0808D906E6E
:101C1A00E0E07002A3E06020123153401B7F0412FF
:101C2A0031247BFF7A16793D1200C9E4906EE0F008
:101C3A00A3F0906F0B7404F0906EDFE0601E123117
:101C4A004D40197F041231247BFF7A16794B12001A
:101C5A00C9E4906EDFF0906F0B7404F0906F0BE0A4
:021C6A00FF2257
:102B8900D201121B7A906FB9EFF06002C201120EE6
:102B990096906FBAEFF06002C20120C60B7BFF7AF4
:102BA9001679581200C9C20120C70B7BFF7A167922
:092BB900691200C9C201A2012247
:10000E00E4FF74B52FF582E4346FF58374FFF00FBF
:05001E00EFB404EE2226
:0C30D400EFC31325E02441FF122F10224F
:1028B300906F0DEFF0E0FFC31325E02441FF7B0190
:1028C3007A6F790F906F157401F0122A5D906F0E75
:1028D300EFF0906F0DE054012402FF74017E00C8F5
:1028E300EFC8088005C333CE33CED8F9FF906F0FFE
:0C28F300E0FDE4EF5D6003D38001C32230
:1028FF00CEEFCEEEC313FF24B5F582E4346FF5832C
:10290F00C083C082E0FDEE5401FC7401C8ECC8081E
:10291F008002C333D8FCF45DD082D083F0EF25E082
:10292F002440FFEEC31324B5F582E4346FAD82FC6F
:08293F007B01D201122ADC2207
:10298F00CEEFCEEEC313FF24B5F582E4346FF5839B
:10299F00C083C082E0FDEE5401FC7401C8ECC8088E
:1029AF008002C333D8FC4DD082D083F0EF25E024D2
:1029BF0040FFEEC31324B5F582E4346FAD82FC7B88
:0729CF0001D201122ADC22F3
:10300400E4F57FFF746D2FF582E4346FF583E4F00B
:063014000FEFB40DEF22E6
:06314D007F50122F10223A
:102F9000906F0FEFF07F507C6F7D0F7B01D201129D
:082FA0002ADC906F10EFF02213
:1027A1007F537B017A6F790C906F157401F0122AB7
:1027B1005D906F0BEFF0A3E0D3941040037410F021
:1027C100906F0CE0FE603A7F517B017A6F799A90AD
:1027D1006F15F0122A5D906F0BEFF0E4F0906F0C23
:1027E100E0FF906F0BE0FE6F6017749A2EF582E4A4
:1027F100346FF583E0FF123114906F0BE004F08029
:02280100DC22D7
:10294700E4906F0FF07F577B017A6F799A906F153C
:102957007410F0122A5D906F10EFF0E4F0906F1092
:10296700E0FF64106017749A2FF582E4346FF583E3
:10297700E0FF12312C906F10E004F080E0906F0FB1
:08298700E004F0E0B408BE22F8
:102F5F00906F0F7442F07F567C6F7D0F7B01D20113
:092F6F00122ADC906F10EFF02231
:102FA800906F06EFF07F547C6F7D067B01C20112A3
:082FB8002ADC906F07EFF02204
:102CCE00C0D075D008906EDFE06022057F906EDE7A
:102CDE00E0657F7018F57F7F557B017A6F7967907D
:102CEE006F15740DF0122A5D906F05EFF0D0D022A3
:10212F00D21DE4F557F558F559906EDEE0FF75F0C6
:10213F000A84755C00F55DEFC313755A00F55B906B
:10214F006EE0E0FEA3E0FF4E6053906F587404F012
:10215F00E4A3F0FCFDF8F9CAEECACBEFCBFF7EC0CB
:10216F007DA81229D67B107A00790078001229D623
:10217F00EF14906F5AF0906F04E075F080A4FF9009
:10218F006EEAE02F906F5BF0906EEDE0906F5CF079
:0E219F007F607C6F7D587B05D201122ADC2206
:063153007F60122F102224
:10254A00C0E0A3E558F0A3E559F0A3E52AF0A3E516
:10255A002CF0A3E52EF0A3E530F0A3E532F0A3E5D5
:10256A0034F0A3E536F0A3E538F0A375F000E529C9
:10257A0042F0E52B232342F0E52DC442F0E52FC4B7
:10258A00232345F0F0A375F000E53142F0E533234B
:10259A002342F0E535C442F0E537C4232345F0F081
:0725AA00A3E540F0D0E022A0
:101F7700C0D075D008906EE0E07002A3E070030255
:101F87002011301D09E5686005E4F557C21DE557C6
:101F9700FB7A00AC5CAD5DFFCEEACE120436ED4CA9
:101FA700705C906EDFE0601DAC5AAD5BCFEBCFCEBF
:101FB700EACE120436ED4C700C906F05741CF0A33A
:101FC7007402F0800A906F05740FF0A37401F0900B
:101FD7006F05E0906F58F0906F06E0906F59F01220
:101FE700254A7F607C6F7D58906F05E0FBC2011228
:101FF7002ADCE56860080559E55970020558055758
:0D200700906EDEE065577002F557D0D022D4
:102E5B000000CC01D8011400F0013C002800E40173
:102E6B00A0016C007800B40150009C018801440063
:050026007EFF7FFF22B8
:1021AD00CBEFCBCAEECAC9EDC9E9540FFFEAEB6F0D
:1021BD00540F25E0FFE433FE745B2FF582EE342ED1
:1021CD00F583EAC4F854F0C868FEEBC4540F48FF19
:1021DD00EE540FFEE4936EFA7401936FFBCFE9CFCB
:1021ED00EFC4540F540FFFEAEF6B540F25E0FFE4DB
:1021FD0033FE745B2FF582EE342EF583EAC4F8546A
:10220D00F0C868FEEBC4540F48FFEE540FFEE49384
:0C221D006EFA7401936FFBCEEACEFF2234
:07313A00EEF4FEEFF4FF22AA
:10280300FF3175FF3100FF310AFF2E3AFF3159FFC7
:102813002DF5FF315FFF3179FF2FC0FF3165FF2EAB
:102823007BFF3043FF317DFF3184FF3185FF3186EC
:10283300FF3187FF3188FF3189FF318AFF318BFFF9
:10284300318CFF318DFF318EFF318FFF3190FF319E
:102853006BFF316BFF316BFF316BFF316BFF316B03
:0F30A000D296D29775D8C575DBECD2BDD2AD22D2
:102F1000E4F56F8F6DD21ED2DDFF122D2CEF6418F9
:0B2F20006004EFB44003D38001C32223
:102ADC00906F11ECF0A3EDF08C838D827880EBFE7F
:102AEC006006E0F6A308DEFA8B6F8F6DD21ED2DD86
:102AFC0030010DCFEBCF122D2C906F13EFF0800522
:0B2B0C00E4906F13F0906F13E0FF22C5
:102A5D00906F12EBF0A3EAF0A3E9F0CEEFCEA3E076
:102A6D00FFF56F8E6DD21ED2DD122D2CE4FE906F10
:102A7D0015E06E601D74802EF8E6FD906F12E0FB80
:102A8D00A3E0FAA3E0F98E82758300ED1204000E27
:032A9D0080DC22B8
:102D2C00CEEFCEE4F56AEE2402FDE433FCE56A6DE9
:102D3C007001EC6010756BDDD56BFD201E03AF6E62
:0B2D4C0022056A80E175D8D57F0022C7
:0431750075D8D52212
:0A310000856DDA75D8C5E4F56C2280
:0A310A00856DDA75D8C5E4F56C2276
:102E3A00C0D075D010E56F700775D8D5C21E800E48
:102E4A00AF6C056C74802FF8E6F5DA75D8C5D0D06A
:012E5A002255
:0631590075D8D5C21E224C
:102DF500C0D075D010E56C656F700775D8D5C21E4B
:102E0500800EAF6C056C74802FF8E6F5DA75D8C5C1
:032E1500D0D022F8
:06315F0075D8D5C21E2246
:0431790075D8E522FE
:102FC000E56F14600A04700C75D8D5C21E800875B0
:082FD000D8C1800375D8C522A9
:0631650075D8D5C21E2240
:102E7B00C0D075D0107480256CF8A6DAE56F1405F8
:102E8B006C656C700575D8C1800375D8C5D0D02220
:10304300C0D075D0107480256CF8A6DA75D8D5C2B7
:043053001ED0D02299
:04317D0075D8D5220A
:013184002228
:013185002227
:013186002226
:013187002225
:013188002224
:013189002223
:01318A002222
:01318B002221
:01318C002220
:01318D00221F
:01318E00221E
:01318F00221D
:01319000221C
:06316B0075D8D5C21E223A
:03002B00022AA006
:102AA000C0E0C0F0C083C082C0D075D01085D96EA0
:102AB000E5D9131313541F75F003A42403F582E41E
:102AC0003428F583E493740193FA740293F912069F
:0C2AD0008DD0D0D082D083D0F0D0E03286
:030000000230E0EB
:0C30E000787FE4F6D8FD7581D70220A8A7
:1003BA00BB010689828A83E0225002E722BBFE0241
:0903CA00E32289828A83E4932274
:1003D300BB010CE58229F582E5833AF583E02250DF
:1003E30006E92582F8E622BBFE06E92582F8E22229
:0D03F300E58229F582E5833AF583E4932243
:10040000F8BB010DE58229F582E5833AF583E8F032
:10041000225006E92582C8F622BBFE05E92582C8DE
:02042000F222C6
:10042200EFF88DF0A4FFEDC5F0CEA42EFEEC88F01F
:04043200A42EFE22D4
:10043600BC000BBE0029EF8DF084FFADF022E4CCAA
:10044600F875F008EF2FFFEE33FEEC33FCEE9DEC73
:10045600984005FCEE9DFE0FD5F0E9E4CEFD22EDB9
:10046600F8F5F0EE8420D21CFEADF075F008EF2F03
:10047600FFED33FD4007985006D5F0F222C398FDF4
:050486000FD5F0EA2291
:10048B00C2D5EC30E709B2D5E4C39DFDE49CFCEE8C
:10049B0030E715B2D5E4C39FFFE49EFE120436C3CA
:1004AB00E49DFDE49CFC800312043630D507C3E4C5
:0604BB009FFFE49EFE22FB
:1004C100C5F0F8A3E028F0C5F0F8E58215827002C6
:0604D1001583E038F02263
:1004D700A3F8E0C5F025F0F0E582158270021583D8
:0604E700E0C838F0E82235
:1004ED00E88FF0A4CC8BF0A42CFCE98EF0A42CFCAE
:1004FD008AF0EDA42CFCEA8EF0A4CDA8F08BF0A42C
:10050D002DCC3825F0FDE98FF0A42CCD35F0FCEB8A
:10051D008EF0A4FEA9F0EB8FF0A4CFC5F02ECD394F
:0F052D00FEE43CFCEAA42DCE35F0FDE43CFC22BC
:10053C0075F008758200EF2FFFEE33FECD33CDCC76
:10054C0033CCC58233C5829BED9AEC99E5829840F9
:10055C000CF582EE9BFEED9AFDEC99FC0FD5F0D6D6
:10056C00E4CEFBE4CDFAE4CCF9A88222B800C1B900
:10057C000059BA002DEC8BF084CFCECDFCE5F0CB3E
:10058C00F97818EF2FFFEE33FEED33FDEC33FCEB77
:10059C0033FB10D703994004EB99FB0FD8E5E4F932
:1005AC00FA227818EF2FFFEE33FEED33FDEC33FC1F
:1005BC00C933C910D7059BE99A4007EC9BFCE99A13
:1005CC00F90FD8E0E4C9FAE4CCFB2275F010EF2F58
:1005DC00FFEE33FEED33FDCC33CCC833C810D70758
:1005EC009BEC9AE899400AED9BFDEC9AFCE899F893
:0E05FC000FD5F0DAE4CDFBE4CCFAE4C8F92226
:1029D600C2D5E830E70FB2D5E4C39BFBE49AFAE42C
:1029E60099F9E498F8EC30E717B2D5122A0C1205DB
:1029F60078E4C39BFBE49AFAE499F9E498F8800337
:102A060012057830D50DE4C39FFFE49EFEE49DFDDC
:042A1600E49CFC221E
:10060A00EB9FF5F0EA9E42F0E99D42F0EC6480C867
:06061A0064809845F02207
:10062000EB9FF5F0EA9E42F0E99D42F0E89C45F030
:0106300022A7
:10063100E8600FECC313FCED13FDEE13FEEF13FFA7
:03064100D8F122CB
:0C064400ECF0A3EDF0A3EEF0A3EFF02229
:10065000A8828583F0D083D08212066712066712C3
:100660000667120667E473E493A3C583C5F0C583E8
:10067000C8C582C8F0A3C583C5F0C583C8C582C8F4
:010680002257
:0C068100A42582F582E5F03583F5832284
:06068D008A838982E473F8
:10005E00E5702433F582E4346FF583E00570229069
:10006E006F30300903906F33E475F0011206B3025E
:10007E0003BA2002E97F2ED2028018EF540F24908B
:10008E00D43440D4FF30060BEF24BFB41A00500313
:10009E002461FFE571600215710574E57470020547
:1000AE007330090E906F30E475F0011206B3EF0253
:1000BE00069302312C7403D2098003E4C209F57051
:1000CE00906F301206CAE4F571F573F574E5716040
:1000DE00077F201200A180F5F572C203C202C2048E
:1000EE00C205C207C208C20A12006DFF700D3009A8
:1000FE00057F001200B2AF74AE7322B42561C2D573
:10010E00C20612006DFF24D0B40A00501C75F00A0E
:10011E0020D50DC571A42571F5717002D20580E050
:10012E00C572A42572F57280D724CFB41A00EF5091
:10013E0004C2E5D2060202ACD20380C4D20280BE53
:10014E00D20480BAD2D580B8D20780B27F201200F6
:10015E00A12004077401B5710040F112005EFF1278
:10016E0000A10200DBD20AD208809312005EFB12BD
:10017E00005EFA12005EF94A4B700679787A037BBC
:10018E00FF200433E571602FAF72BF00011F7E00A8
:10019E008E827583001203D360050EEE6F70F1C26E
:1001AE00D5EBC0E0EAC0E0E9C0E0EE1202F0D0E02C
:1001BE00F9D0E0FAD0E0FB1203BAFF60A5EBC0E085
:1001CE00EAC0E0E9C0E01200A1D0E02401F9D0E0DD
:1001DE003400FAD0E0FBE57260DDD572DA80837B05
:1001EE00FF7A0279ECD2048098791080027908C2E5
:1001FE0008C20A8008D2D5790A8004790AC2D5E4E9
:10020E00FAFDFEFF12005EFC7B0820031312005E57
:10021E00FD7B1030020A12005EFE12005EFF7B2094
:10022E00EC3382D592D55013C3E43002069FFFE41F
:10023E009EFEE42003039DFDE49CFCE4CBF8C20388
:10024E00EC700CCFCECDCCE824F8F870F38017C349
:10025E00EF33FFEE33FEED33FDEC33FCEB33FB9966
:10026E004002FB0FD8E9EB300305F8D0E0C448B2EA
:10027E0003C0E00AEC4D4E4F78207B0070C2EAC0FE
:10028E00E01202F2D0F0D0E0200304C4C0E0C4B209
:10029E0003C0F012008AD0F0D5F0EB0200DB12069C
:1002AE00D301795301F758014A4C01464201FB4FE5
:1002BE00020344020349015F4302095501ED460161
:1002CE00ED4501ED47039B50014E2D01522E017558
:1002DE002B01562301732003862A0000016D3F3F38
:1002EE003F00790AA2D5200514300709B91002047F
:1002FE0004B9080104A2D5200802500104200466A6
:02030E00920457
:10031000B571005032C0E07F203005177F30A20455
:1003200072087207500D120347C204C208C2077F49
:1003300030800F300703E9C0E01200A1300703D07E
:10034000E0F9D0E0B571CE3007177F30B9100C124C
:1003500000A17F583006077F788003B90803120098
:10036000A13004057F2D0200A17F20200AF87F2BF9
:100370002008F322920480CF286E756C6C29002D22
:1003800050434958D20312005E3003F8C20378711B
:1003900030D504D2027872F602010C12005E2403FA
:1003A000B405004001E490037F93120092743A1266
:0A03B0000092D2057571040201F7F6
:10301A00EFC394094006EFC3940E4004EFB42003B3
:05302A00D38001C32268
:102DA900EFC394414006EFC394474018EFC39461C1
:102DB9004006EFC39467400CEFC394304009EFC35A
:092DC900943A5003D38001C322A7
:1025B100906F0FEBF0A3EAF0A3E9F0906F12E0FB4C
:1025C100A3E0FAA3E0F91203BAFE906F0FE0FBA3B8
:1025D100E0FAA3E0F91203BAFD6E702AED600E90E5
:1025E1006F1574FFF5F01204C145F070037F0022EE
:1025F100906F10E475F0011204C1906F13E475F04F
:10260100011204C180B5D3EE6480F8ED6480984076
:07261100037F01227FFF227D
:102EF400E94A4B7001221203BAFF6D700122EF7090
:0C2F040004FBFAF92209E970ED0A80EAEA
:10167800906F29EBF0A3EAF0A3E9F0906F29E0FB63
:10168800A3E0FAA3E0F91203BAFF12301A500C9043
:101698006F2AE475F0011204C180E0D201906F292D
:1016A800E0FBA3E0FAA3E0F91203BAFF642B60049D
:1016B800EFB42D1D906F29E0FBA3E475F00112042F
:1016C800D7A9F0FA1203BA642D6003D38001C3923C
:1016D80001906F2C12065000000000906F29E0FB6B
:1016E800A3E0FAA3E0F91203BAFF12308F506A7F21
:1016F8000A7E007D007C00906F2CE0F8A3E0F9A33F
:10170800E0FAA3E0FB1204EDC8ECC8EDC0E0EEC0BF
:10171800E0EFC0E0906F29E0FBA3E0FAA3E0F91244
:1017280003BAFF3395E0FEEF24D0FFEE34FFFEE46A
:10173800FCFDD0E0FBD0E0FAD0E0F9EB2FFFEA3E69
:10174800FEED39FDEC38FC906F2C120644906F2AA0
:10175800E475F0011204C18082300110906F2CE012
:10176800FCA3E0FDA3E0FEA3E0FF8011906F2CE056
:0E177800FCA3E0FDA3E0FEA3E0FF1206A52205
:10069300BB010689828A83F0225002F722BBFE0146
:0206A300F32240
:0E06A500C3E49FFFE49EFEE49DFDE49CFC2266
:1006B300F8E0FBA3A3E0F925F0F0E58215827002D0
:0706C3001583E0FA38F02274
:0906CA00EBF0A3EAF0A3E9F02231
:1006D300D083D082F8E4937012740193700DA3A3B6
:1006E30093F8740193F5828883E4737402936860CA
:0606F300EFA3A3A380DFCA
:10308F00EFC394304009EFC3943A5003D38001C388
:01309F00220E
:00000001FF
